:100000000110060000000000601C0000FF0000005E
:10001000020BD7FFFFFFFFFFFFFFFF0216137E0358
:100020009000BEE06F6007EFF0E49000C1F0900038
:10003000BEE07001FE9000C1E004F0C39E50037F5B
:1000400000229000C17403F07F012202178EE4FBAE
:10005000EB25E025E024ADF812025DEB25E025E07C
:1000600024BDF81202760BBB04E622020F30BB015E
:100070000689828A83E0225002E722BBFE02E32245
:1000800089828A83E49322EF8DF0A4A8F0CF8CF0CC
:10009000A428CE8DF0A42EFE22BC000BBE0029EFBA
:1000A0008DF084FFADF022E4CCF875F008EF2FFF5F
:1000B000EE33FEEC33FCEE9DEC984005FCEE9DFE2D
:1000C0000FD5F0E9E4CEFD22EDF8F5F0EE8420D274
:1000D0001CFEADF075F008EF2FFFED33FD400798E3
:1000E0005006D5F0F222C398FD0FD5F0EA22BB01ED
:1000F0000A89828A83E0F5F0A3E022500687F0099E
:10010000E71922BBFE07E3F5F009E3192289828A89
:1001100083E493F5F074019322E88FF0A4CC8BF084
:10012000A42CFCE98EF0A42CFC8AF0EDA42CFCEAB3
:100130008EF0A4CDA8F08BF0A42DCC3825F0FDE9ED
:100140008FF0A42CCD35F0FCEB8EF0A4FEA9F0EBE3
:100150008FF0A4CFC5F02ECD39FEE43CFCEAA42DEF
:10016000CE35F0FDE43CFC2275F008758200EF2FDF
:10017000FFEE33FECD33CDCC33CCC58233C5829B6D
:10018000ED9AEC99E58298400CF582EE9BFEED9A93
:10019000FDEC99FC0FD5F0D6E4CEFBE4CDFAE4CC2F
:1001A000F9A88222B800C1B90059BA002DEC8BF031
:1001B00084CFCECDFCE5F0CBF97818EF2FFFEE33EE
:1001C000FEED33FDEC33FCEB33FB10D70399400419
:1001D000EB99FB0FD8E5E4F9FA227818EF2FFFEE40
:1001E00033FEED33FDEC33FCC933C910D7059BE971
:1001F0009A4007EC9BFCE99AF90FD8E0E4C9FAE4CD
:10020000CCFB2275F010EF2FFFEE33FEED33FDCC6B
:1002100033CCC833C810D7079BEC9AE899400AED55
:100220009BFDEC9AFCE899F80FD5F0DAE4CDFBE4FD
:10023000CCFAE4C8F922EB9FF5F0EA9E42F0E99D82
:1002400042F0E89C45F022E8600FECC313FCED138C
:10025000FDEE13FEEF13FFD8F122E8600FEFC3337A
:10026000FFEE33FEED33FDEC33FCD8F122E6FC0863
:10027000E6FD08E6FE08E6FF22E6FB08E6F908E6EA
:10028000FA08E6CBF822ECF608EDF608EEF608EFF1
:10029000F622ECF208EDF208EEF208EFF222D0833B
:1002A000D082E493F608740193F608740293F6087A
:1002B000740393F6740473D083D082E493F20874C9
:1002C0000193F208740293F208740393F2740473B6
:1002D0008A838982E4738E568F57E4F559F55AF56F
:1002E0005B9000D1E0F55AA3E0F55BE4F55890008F
:1002F000BFE070139000C1E0B4030CD37895E29492
:100300000018E29400401EE55825E02484F8E4F249
:1003100008F2E55825E025E0246CF81202A7000059
:1003200000000203DCE55825E02485F9E37002199A
:10033000E3701AE55825E02400F8E2FE08E2FFE544
:100340005825E0247CF8EEF208EFF28057E55825B6
:10035000E0247CF8E2FE08E2FFE55825E02400F8FE
:10036000E2FC08E2FD121B21D3EF955BEE955A40AB
:1003700033E55825E02400F8E2FE08E2FFE55825C1
:10038000E0247CF8EEF208EFF2E55825E02484F84A
:10039000E4F208F2E55825E025E0246CF81202A703
:1003A00000000000E55825E02400F8E2FE08E2FF26
:1003B000E55825E025E0246CF8C000E2FB08E2F9EE
:1003C00008E2FA08E2CBF8E4FCFDEB2FFFEA3EFE80
:1003D000ED39FDEC38FCD000120282E55825E0240E
:1003E00084F808E22401F218E23400F20558E558D6
:1003F000C3940450030202DEE4F558E55825E024D6
:1004000085F9C3E3955719E39556400205590558F8
:10041000E558B404E6E559640460030204D674FFA9
:100420009000D3F0A3F0E4A3F0A3F0F558E558252D
:10043000E02484F8E2FE08E2FF4E70030204B9E40F
:10044000FCFDC004A905AA06AB07E55825E025E098
:10045000246CF8E2FC08E2FD08E2FE08E2FFD000AE
:100460001201948E5C8F5DD39000D4E0955D900076
:10047000D3E0955C4007E55CF0A3E55DF0C3900038
:10048000D6E0955D9000D5E0955C5007E55CF0A363
:10049000E55DF0E55825E02408F8E55CF208E55D47
:1004A000F2E55825E02484F8E4F208F2E55825E066
:1004B00025E0246CF81202A700000000C2080558CD
:1004C000E5586404600302041D9000D3E0FEA3E03D
:1004D000FFA3E0FCA3E0FD121B21D3EF9464EE9494
:1004E00000400312173722E4F554E55425E025E0D7
:1004F00024BDF8C00012025DC00774732554F8E6ED
:10050000FFFBE4FAF9F8D007120109D000120276D5
:10051000E55425E025E024BDF8C00012025D78070F
:10052000120237D000120276E55425E025E024BD02
:10053000F812025DEC4D4E4F6076E55425E025E063
:10054000249DF812025DE55425E025E024BDF81253
:100550000269C312022650037F0322E55425E025D9
:10056000E0249DF8120269C000E55425E025E0244E
:10057000BDF812025DD000C3EF9BF558EE9AF55717
:10058000ED99F556EC98F555E47FFF7EFFFDFCAB49
:1005900058AA57A956A855C312022640037F032222
:1005A000E55425E02400F8E557F208E558F28015F7
:1005B000E554C39404500BE55425E02410F8E4F20C
:1005C00008F27F03220554E554640460030204DA50
:1005D000E4F554E55425E02408F8E2FE08E2FFE5DE
:1005E0005425E02400F8E2FC08E2FDD39FEC9E4095
:1005F0001EE55425E02408F8E2FE08E2FFC3ED9F63
:10060000FFEC9EFEE48F5C8E5BF55AF5598009E4A1
:10061000F55CF55BF55AF559E554C39404506DAF9C
:100620005CAE5BAD5AAC59780712024A8F5C8E5BA8
:100630008D5A8C59E55425E025E02440F8E2FC0869
:10064000E2FD08E2FE08E2255CFFEE355BFEED35DB
:100650005AFDEC3559FC7801120237E55425E025A6
:10066000E02440F8120282E55425E025E02440F819
:10067000E2FC08E2FD08E2FE08E2FF78071202371A
:10068000E55425E02410F8EEF208EFF20554E554A5
:10069000640460030205C37F0722E4F557F556E5BD
:1006A0005625E025E0246CF81202A70000000005A2
:1006B00056E556B404E91218C3E4F556E55625E0AC
:1006C00025E0246CF8C000E2FC08E2FD08E2FE0828
:1006D000E2FFE55625E025E024ADF8120269EF2B94
:1006E000FFEE3AFEED39FDEC38FCD0001202820537
:1006F00056E556B404C60557E557C3940540B7E41C
:10070000F556AF57E4FCFDFEC004A905AA06AB07E9
:10071000E55625E025E0246CF8E2FC08E2FD08E25D
:10072000FE08E2FFD0001201948F5B8E5A8D598C27
:1007300058AB5BAA5AA959A858C00074732556F83B
:10074000E6FFE4FCFDFED0001201098F5B8E5A8D9E
:10075000598C5878071202378F5B8E5A8D598C58F6
:10076000E47FE87E03FDFCAB5BAA5AA959A858D3E5
:100770001202264030E55B2418FFE55A34FCFEE502
:100780005934FFFDE55834FFFCE55625E025E0240B
:100790009DF8120276E55625E02400F87403F2086D
:1007A00074E8F2801EE55625E025E0249DF812024B
:1007B0008E00000000E55625E02400F8E55AF20816
:1007C000E55BF2E55625E025E0246CF81202A7006F
:1007D000000000E55625E02484F8E4F208F2E5562E
:1007E000C394045033E55625E02400F8E2FE08E205
:1007F000FFE55625E02408F8EEF208EFF2E556256D
:10080000E02410F8E4F208F2E55625E025E0244063
:10081000F81202A7000000000556E55664046003C4
:100820000206F22285BA5C53BA0F43BA10E4F556B9
:10083000E55625E025E024ADF812028E0000000008
:100840000556E556B404E975560575ABFF121A4115
:10085000E4F557E55725E025E024ADF8C000120285
:100860005DC004C005C006C00774CD2557F8E67505
:10087000F003A4243BF582E4341BF583E493FB747A
:100880000193FA740293F91202C0A804A905AA06FA
:10089000AB07D007D006D005D004EF2BFFEE3AFE11
:1008A000ED39FDEC38FCD0001202760557E557C350
:1008B0009404409FE4F5AB121A41E4F557E557253F
:1008C000E025E024ADF8C00012025DC004C005C000
:1008D00006C00774CD2557F8E675F003A4243BF550
:1008E00082E4341BF583E493FB740193FA7402935E
:1008F000F91202C0A804A905AA06AB07D007D006C2
:10090000D005D004C3EF9BFFEE9AFEED99FDEC9865
:10091000FCD0001202760557E557C39404409E159B
:1009200056E556600302083AE4F557E4755B107526
:100930005A27F559F558AF5BAE5AAD59AC58780700
:1009400012024A8F5B8E5A8D598C58E55725E02547
:10095000E024ADF81202691201948F5B8E5A8D5912
:100960008C5874732557F8A6070557E557B404BB90
:10097000855CBA2230040E755700755814755900FD
:10098000755A3C800C755700755814755900755A86
:100990003CE4FDED25E02458F8E2FE08E2FFED25F9
:1009A000E02419F9D3E39F19E39E4016ED25E024D6
:1009B00018F8E2FE08E2FFED25E02458F8EEF20810
:1009C000EFF2EDC39402506AE557C313FEE55813E6
:1009D000FFED25E02419F9D3E39F19E39E5023EDA1
:1009E00075F008A4247DF8A65708A658E55825E018
:1009F000FFE55733F8ED25E02458C8F208EFF2027E
:100A00000A86ED25E02419F9D3E3946419E39400F0
:100A10005003020A86ED25E02458F9E3C313FE09CA
:100A2000E313FFED75F008A4247DF8A60608A607D9
:100A30008064E559C313FEE55A13FFED25E0241940
:100A4000F9D3E39F19E39E5022ED75F008A4247DAD
:100A5000F8A65908A65AE55A25E0FFE55933F8EDFE
:100A600025E02458C8F208EFF2802BED25E0241988
:100A7000F9D3E394C819E39400401BED25E0245812
:100A8000F9E3C313FE09E313FFED75F008A4247D19
:100A9000F8A60608A6070DED64046003020983E4C6
:100AA000FDED75F008A4247DF8E6FE08E6FFED25CF
:100AB000E02460F8EEF208EFF20DBD04E42220CA53
:100AC00003020BD67862E67003020BD6E4786CF66C
:100AD000F55474622554F8E6FF744A2554F8A607C5
:100AE00074622554F8E4F60554E554B40AE4786CCD
:100AF000E6700320CA12E4F554744A2554F8E4F66B
:100B00000554E554B40AF222E54A24E0601F24F0BB
:100B1000602224F0604224F0606224F0606624F0D9
:100B2000606A2460706FE4FF121AAD80687F011262
:100B30001AAD8061787D7600087614788576000895
:100B40007614788D760008763C7895760008763CA9
:100B50007870E64410F6803D787D7600087614784B
:100B6000857600087614788D760008763C78957640
:100B70000008763C7870E654EFF680197870E64409
:100B800001F680117870E654FEF68009E4FF121B2E
:100B90007C7872A607E54A54F064807049E54B45BD
:100BA0004C6043E54BFE7C00E4254CFFEC3EFEC36D
:100BB000EF940AEE9400402EE54A540FFDBD0F1944
:100BC000E4F554E55475F008A4247DF8A60608A6BB
:100BD000070554E554B404EB22ED75F008A4247D18
:100BE000F8A60608A60722439F04E453C6DFE5C61D
:100BF00000B5C6F375830075820775FD0DE4E5FE4B
:100C0000F4FF75830075820675FD0DE4E5FEB507FA
:100C100004F59E8003759E0078100000D8FC53C632
:100C2000E043C60843C68075960575970375830033
:100C300075820475FD0D85FE8F75830075820375C1
:100C4000FD0DE4E5FEF4FF75830075820275FD0D70
:100C5000E4E5FEB50704F595800375958375BE0E32
:100C60005392FE9001007F007E02E4F0A3DFFCDEE1
:100C7000FA78007F00E4F208DFFC78FFE4F6D8FDA4
:100C80007581D8020CB4020000021014E493A3F89A
:100C9000E493A34003F68001F208DFF48029E49393
:100CA000A3F85407240CC8C333C4540F4420C8838A
:100CB0004004F456800146F6DFE4800B010204088C
:100CC00010204080901539E47E019360BCA3FF544E
:100CD0003F30E509541FFEE493A360010ECF54C0DA
:100CE00025E060A840B8E493A3FAE493A3F8E49362
:100CF000A3C8C582C8CAC583CAF0A3C8C582C8CA6A
:100D0000C583CADFE9DEE780BE7557FF30040B7587
:100D10003B00753C00753D338009753B00753C0018
:100D2000753D2BE4F55CAB3BE53DF92402F53DE573
:100D30003CFA3400F53C1200DEFFE55C25E0243E81
:100D4000F8A6F008A607055CE55CB404D9E4F55CF8
:100D5000E55C25E0243EF8E6FE08E6FFE55C25E0DC
:100D60002411F9C3E39F19E39E4003020E09E55CD9
:100D700025E02442F8E6FE08E6FFE55C25E02414C1
:100D8000F8E2FC08E2FDC39FEC9E4003020E09E579
:100D90005C7020E55C25E02410F8E2FE08E2FF2408
:100DA00028F55BE43EF55AEF24FBF559EE34FFF5E8
:100DB000588021E55CB4011C25E02410F8E2FE080F
:100DC000E2FF2414F55BE43EF55AEF24EAF559EE10
:100DD00034FFF558C3ED955BEC955A5008ED9559E5
:100DE000EC95585011E55C25E02411F9C3E3940A11
:100DF00019E394005023AF5C7401A807088002C374
:100E000033D8FCF45257E55C2402FF7401A80708AC
:100E10008002C333D8FCF45257055CE55C64026081
:100E200003020D40855724227556077D0774017E05
:100E300000A856088005C333CE33CED8F9FFACAC3A
:100E4000ECFBE4EF5B7003D556E3ED601D74017EAF
:100E500000A805088005C333CE33CED8F9FFACAE69
:100E6000ECFBE4EF5B70031D80E0AF567401A80754
:100E7000088002C333D8FCF5AC7401A805088002D1
:100E8000C333D8FCFFF5AD8FAE53AACF85BA5F53FD
:100E9000BA0F43BA10E4F55AF559F558F557121A36
:100EA00041E4F55674CD2556F8E675F003A4243BCD
:100EB000F582E4341BF583E493740193FA7402938E
:100EC000F91202C08F5E8E5D8D5C8C5BAB5AAA59A5
:100ED000A958A857C3120226500C855E5A855D5941
:100EE000855C58855B570556E556C3940440B5AFFD
:100EF0005AAE59AD58AC577802120237E55A2FF561
:100F00005AE5593EF559E5583DF558E5573CF55732
:100F1000AF5AAE59AD58FC78101202378FB3AF5AA2
:100F2000AE59AD58AC5778081202378FB2855AB116
:100F300043AA30855FBA75AC0375ADC075AEC022EB
:100F4000C0E0C0F0C083C082C0D075D008C2CF302E
:100F5000CD0302100930CB4720CC447861A6CEE601
:100F6000FFC39480403075F003EFA424FEF582E5C2
:100F7000F03414F583E493FB740193FA7402938BB9
:100F8000478A48F5490549E5497002054814F912B0
:100F9000005EF5CE80097861E62546F8E6F5CE30AC
:100FA000CC297861E6C394804015AB470549E549F3
:100FB000AA487002054814F912005EF5CE805678F2
:100FC0006106E62546F8E6F5CE804A20CB47AFCE4F
:100FD0007861E6FE702EBF100553803F8037BF203A
:100FE000054380C0802FBF50087870E64401F6802A
:100FF00024BF60087870E654FEF680197862A60F68
:1010000018068011EEC3940A50087861E62462F84D
:10101000A60F786106786C7601D0D0D082D083D0CC
:10102000F0D0E032121AE97D01E4FF12196E7F015F
:10103000121AAD7F01121ACC121C35121C28121A7A
:10104000671215A81219A4121A0DD2AF751C01E56A
:101050001C24FD601114601924FE602614602A14FB
:1010600060702407706F1218341214BC751C048051
:1010700064D2D8E51D70FC12003E121B53751C068D
:1010800080531204D78F1C804CD39000C7E094008B
:101090009000C6E09400400CA3E024FFF09000C64E
:1010A000E034FFF0D37895E2940018E29400400A0F
:1010B00008E224FFF218E234FFF29000C3E004F0EB
:1010C00070069000C2E004F01212721210F78F1C2A
:1010D0008003751C049000D7E0B40124E4786CF61A
:1010E000FF121C35E4F0F518F519000519E5197023
:1010F000020518B42CF4E518B401EF7F01121C3579
:10110000120AAE02103F22E4F55475550812131965
:1011100012187F1213B11218FF9000BFEFF01200E7
:101120000EEF60557F011219D9AD07AC06D39000C0
:10113000C7E094009000C6E09400400FED7802CE26
:10114000C313CE13D8F9FDAC068025300811EDAEDF
:10115000047803CEC313CE13D8F9FDAC068011205A
:10116000090EECC4F854F0C868FCEDC4540F48FDF7
:10117000AF05AE041202C68003AF55229000BEE058
:10118000F554E5546034E49000CAF0A3F09000C92F
:10119000E004F070069000C8E004F07F051219D951
:1011A000D39000C9E09F9000C8E09E4014E4FF1275
:1011B00016DBE49000C0F07F0322E49000C8F0A3A7
:1011C000F09000C0E06554600BAF541216DB900045
:1011D000C0E554F0AF55227DFFE522700302126C8A
:1011E0007824E2FE08E2FF7821E22FF55818E23E6B
:1011F000F5577826E2FE08E2FF7823E22FF55A1829
:10120000E23EF559787EE625E0FF18E633FEC37826
:1012100021E29F18E29E4014788EE625E0FF18E652
:1012200033FEC37825E29F18E29E5013E559C3139D
:10123000FEE55A13D39558EE955740035305FA78B7
:1012400086E625E0FF18E633FEC37823E29F18E226
:101250009E40147896E625E0FF18E633FEC3782713
:10126000E29F18E29E5018E557C313FEE55813D3CA
:10127000955AEE955940085305F580035305F08DB6
:101280002322E4F55430091AE55475F008A4247FAC
:10129000FFE55425E02418F8E2FC08E2FD121B6883
:1012A000801DE55475F008A4247FFBE55425E02457
:1012B00018F9E3C313FC09E313FDAF03121B68E540
:1012C0005475F008A42481FFE55425E02410F8E2C9
:1012D000FC08E2FD121B68E55475F008A42483FBAA
:1012E000C003E55425E02400F8E2FE08E2FFE4FC38
:1012F000FDE55425E025E0249DF8120269EF2BFF5F
:10130000EE3AFEED39FDEC38FC7804120237AD07F9
:10131000AC06D007121B680554E554C3940450036F
:101320000212757870E6F52022E4F556E55625E0C0
:101330002410F8E2F55708E2F558AE57FFE4FCFD3B
:101340007B64FAF9F8120109C006C007E55625E0EA
:101350002496F582E43400F583E0FEA3E0FFFBAAC7
:1013600006E4F9F8D007D006120194E55625E024EA
:1013700020F8EEF208EFF2AE57AF58E4FCFD7B64C4
:10138000FAF9F8120109C006C007E55625E02496CF
:10139000F582E43400F583E0FEA3E0FFFBAA06E457
:1013A000F9F8D007D006120194E55625E02418F884
:1013B000EEF208EFF20556E5566404600302131CD2
:1013C00022E4F556E55625E02408F8E2FE08E2FF9F
:1013D000E55625E02400F8E2FC08E2FDC39FEC9E00
:1013E0005048E55625E02409F8C3E29DF55818E277
:1013F0009CF557FEAF58E4FCFD7B64FAF9F8120146
:1014000009C006C007E55625E02496F582E43400BD
:10141000F583E0FEA3E0FFFBAA06E4F9F8D007D0CD
:10142000061201948E598F5A8009E4F557F558F544
:1014300059F55AD3E55A940AE55994004002D20866
:101440000556E556640460030213B422E4FFFEEE81
:1014500075F008A4247DF8E6FC08E6FDEE25E024FE
:1014600021F9C3E39D19E39C401DEE25E02425F9F5
:10147000C3E3940A19E39400400D7401A8060880A0
:1014800002C333D8FC4207EE75F008A4248DF8E6B9
:10149000FC08E6FDEE25E02425F9C3E39D19E39C55
:1014A0004021EE25E02421F9C3E3940A19E39400D6
:1014B0004011EE2402FD7401A805088002C333D850
:1014C000FC42070EEE640270868F2222E4F554F58A
:1014D00055121B06E49000BEF09000C0F0A3F090FF
:1014E00000C8F0A3F0A3F0A3F09000DAF0A3F07826
:1014F00094F208F2F521FFEF25E02496F582E4341A
:1015000000F583E0FCA3E0FD9000D2E02DF0900018
:10151000D1E03CF00FBF02DF9000D1E0FEA3E0FF7E
:101520007C007D0A1200899000D1EEF0A3EFF0124A
:101530000E1812081412068A7F0A1219D99000C6D2
:10154000EEF0A3EFF0121B5322082B0050005A00BC
:1015500078006E08330050005A0078006E08CD0302
:101560000104020706FFFF04D500000000604600EA
:1015700096014001EA008200BE0046004600460097
:1015800046010204080506070800000000000000EC
:10159000000000000000000000000000000000004B
:1015A000000000000000000000000000000000003B
:1015B0000000000000000000E4F554786DF6FF1212
:1015C0001B7C8F54E554BFFF06786E760680047846
:1015D0006E76FF786F7605E408F6787276FF787D90
:1015E000F60876147885F6087614788DF608763C39
:1015F0007895F608763CFFEF75F008A4247FF8E4B0
:10160000F608F6EF75F008A42481F8E4F608F6EF82
:1016100075F008A42483F8E4F608F60FBF04D87523
:10162000466D22C0E0C0F0C083C082C0D075D0003B
:10163000C000C004C005C006C007C28D758CD87537
:101640008AF0051BE51B7002051AAE1AFF7C007DAF
:1016500064120089ED4C70219000C2E0FEA3E0FF0F
:10166000D3940AEE94004006A3EEF0A3EFF09000AE
:10167000C2E4F0A3F0F51AF51BD007D006D005D0D0
:1016800004D000D0D0D082D083D0F0D0E032FE00A1
:1016900000FE0008FE0008FE0010FE0010FE00180C
:1016A000FE0018FE0020FE0020FE00280000AD0015
:1016B00000B50000BD0000C5FE0000FE0008FE00F1
:1016C00050FE00400100C20000220100BE0100D512
:1016D0000100C00100D7FE00940100AE0100B60178
:1016E00000BFFE0058FE0060FE00849000D7E0704E
:1016F0005504F0E4FEFDFC7401A804088002C33325
:10170000D8FCF9FB9000C0E05BB50313EC2404FAAD
:101710007401A802088002C333D8FC42068003E9A2
:101720004206EF5BB50305E942058011EC2404FB9A
:101730007401A803088002C333D8FC42050CBC0224
:10174000B6EE5D786DF622E4FBEB25E025E024BDE6
:10175000F812025DEF2418FFEE34FCFEED34FFFDBD
:10176000EC34FFFCEB25E025E0249DF8120276EB3B
:1017700025E02400F87403F20874E8F2EBC3940443
:101780005017EB25E02410F8E4F208F2EB25E024F2
:1017900008F87403F20874E8F20BBB04AC22C0E052
:1017A000C0F0C083C082C0D075D01053B9FD756041
:1017B0000074CD2560F8E675F003A4243BF582E4BF
:1017C000341BF583E493740193FA740293F91202C3
:1017D000C0E56025E025E024ADF81202760560E55D
:1017E00060C3940440CB751D00D0D0D082D083D08C
:1017F000F0D0E032A907E4FDFC74017E00A80408E3
:101800008005C333CE33CED8F9FFE9FB7A00EAEF87
:101810005B701DEC2402FF74017E00A807088005A0
:10182000C333CE33CED8F9FFEE5AFEEF5B4E600DD8
:101830007401A804088002C333D8FC42050CBC0222
:10184000B8AF0522E4FFFE74CD2EF8E6901C3E935F
:1018500042070EBE04F1EF42D4EF42F4EF42E4EF50
:10186000F452DC75AA3B75BA0C43BA4043B9205315
:10187000B9BF8FB4E4F5B375B24E75B12075BBFF37
:1018800075A950F5AB75AC0375ADC075AEC02278C7
:1018900020E2FE08E2FF8E56F5577D01ED25E0249B
:1018A00020F8E2FA08E2FBC39557EA955650048AFD
:1018B000568B57D3EB9FEA9E4004AE02AF030DBD9B
:1018C00002DA786AE556F208E557F27868EEF2082F
:1018D000EFF222121A41E4F55C74CD255CF8E6754E
:1018E000F003A4243BF582E4341BF583E4937401F4
:1018F00093FA740293F91202C0E55C25E025E02416
:10190000ADF8120276055CE55CC3940440CB22126C
:10191000096412143C1211C7120CF9121938900004
:10192000BEE0700D852256E5235256E524525680BE
:1019300007852556E5235256E5566004D2098002F4
:10194000C209AF561217E422E4FFFEEE75F008A4B8
:10195000247EF8E624FBFD18E634FFFCEE25E024A7
:1019600019F9C3E39D19E39C400D7401A806088092
:1019700002C333D8FC42070EBE04D08F2522E4FEFA
:101980007C0474CD2CF8E6901C3E9342060CBC06F9
:10199000F1EF6005EE42D48004EEF452D4EEF4FF91
:1019A00052F4EE42E4ED6005EE42EC8003EF52ECBF
:1019B000EF52DC227E007FAEE4FDED25E0248DF5C4
:1019C00082E4341AF583E493F4601DED25E0248E5F
:1019D000F582E4341AF583E493FCEF2DF582E43EBE
:1019E000F583ECF00DBD10D2227556007557AE7B15
:1019F000017A00BFFF057F017E0022E5572FF582A7
:101A0000E43556F583E07A00FB9000C4E0FCA3E0E7
:101A1000FDAF037E00120077AA06AB072243F80849
:101A200075CD4053CC7F43CC4043CC2043CC1043B6
:101A3000CC0453CCFD43CB0243CB0153CBBF43E893
:101A40000853E5FC43E30243F50343900343ED03EE
:101A50002275BF0F00000000000000000000000021
:101A6000000000000000D2D853B9FD43B901E5B928
:101A700030E1FBE4F5BF22438901C28DD2A953B8FE
:101A8000FDE4F51AF51B9000C2F0A3F0A3F0A374D7
:101A900064F0758CD8758AF0D28CD2AF2200020126
:101AA00001020103010405050606060702080A09EA
:101AB000020A020B280C010D030E01FF01E4FE7D5A
:101AC0000474CD2DF8E6901C3E9342060DBD06F140
:101AD000EF6004EE428022EEF4528022EF60054374
:101AE000D504800353D5FB53F5FB53E5FB43E304D7
:101AF00043ED04E49000D7F022E4F5E3439F104364
:101B00009F02FF0FBFFFFC539FEF75BE0EE4F5BFB2
:101B1000F5B97592762253BAFEE5B920E004E51DC9
:101B20006005E5B930E1FBE4F5BF53B9FE53B9FDFB
:101B300022AB07AA06D3EB9DEA9C4007EB9DFFEA88
:101B40009CFE22C3ED9BFFEC9AFE22FF1B90FF1B25
:101B5000A3FF1BB6FF1BC9FF1BDCFF1BEFFF1C0213
:101B6000FF1C1575BF0F43B92053B9FD43BA01756A
:101B70001D0143B901D2D822AB07AF04AE05C2AFF5
:101B8000A803A607E804F8A606D2AF22E4FFF58270
:101B9000F5837420FEE493F42FFFA3EEB583F622C1
:101BA00053B9EF78D6A6B708A6B608A6B578D51269
:101BB000025D2253B9EF78D6A6EB08A6EA08A6E99B
:101BC00078D512025D2253B9EF78D6A6F308A6F2B3
:101BD00008A6F178D512025D2253B9EF78D6A6FB9C
:101BE00008A6FA08A6F978D512025D2243B9107842
:101BF000D6A6B708A6B608A6B578D512025D2243C8
:101C0000B91078D6A6EB08A6EA08A6E978D512029C
:101C10005D2243B91078D6A6F308A6F208A6F1789B
:101C2000D512025D2243B91078D6A6FB08A6FA08A1
:101C3000A6F978D512025D22C2DA53D80F43D8D064
:101C4000D2D8D2D922EF6003D29222C292220102CC
:101C5000040810204080DFFFFFFFFFFFFFFFFFFFB2
:101C6000FFFFFFFFFFFFFFFFFFFFFFFFFFFFFFFF84
:00000001FF
